:1000000019C033C032C031C030C02FC02EC02DC087
:100010002CC02BC02AC02AC028C027C026C025C09B
:1000200024C023C022C021C020C01FC01EC01DC0CC
:100030001CC01BC011241FBECFEFD4E0DEBFCDBF5C
:1000400011E0A0E0B1E0E0EAF4E002C005900D921A
:10005000A631B107D9F721E0A6E1B1E001C01D92B8
:10006000A731B207E1F7BFD019C2CACF1F920F92D2
:100070000FB60F9211248F939F93EF93FF9315B8B0
:100080001BB88DE08A95F1F7000081E090E00090C8
:10009000160102C0880F991F0A94E2F785B9E09112
:1000A0001601F0E0E050FF4FE081F0E0ED5FFE4F21
:1000B00080818BB9809116018F5F833018F4809313
:1000C000160102C010921601FF91EF919F918F913E
:1000D0000F900FBE0F901F9018958FEF8AB987E091
:1000E00084B9109280008AE08093810084EC99E0CA
:1000F0009093890080938800EFE6F0E08081826031
:100100008083789408959DEC899F912D1124969574
:1001100096959695E0E0F1E09283990F292F220FB2
:10012000220F920F891B81836083089543983B9A25
:100130008FE599E00197F1F700C000003B98EBE2F2
:10014000F1E03197F1F700C0000086B1E3E3F8E099
:100150003197F1F700C000008870089543983B9AEA
:1001600096E09A95F1F700C0813009F43B988BE254
:1001700091E00197F1F700C000003B980895CF93FC
:10018000DF93D82FC8E08D2F8170E8DFD695C1505E
:10019000D1F7DF91CF91089543983B9A86E08A95F5
:1001A000F1F700C03B98EDE5EA95F1F7000086B164
:1001B000E0EEF0E03197F1F700C0000083FB882704
:1001C00080F90895CF93DF93D8E0C0E0E5DF20E821
:1001D000829FC0011124C695C82BD150B9F78C2F2E
:1001E000DF91CF91089579DFE0E0F1E081E1828352
:1001F000818380832FEF8BE792E9215080409040EC
:10020000E1F700C0000092DF8CECB9DF84E4B7DFD7
:10021000C3DF8823E9F38ADF8CECB1DF8EEBAFDF3D
:10022000D1DFC82FCFDF682F70E0762F66276C0FE5
:10023000711D072E000C880B990B41D020E030E097
:1002400040E85DE3A0D00DD0862F6EE05CDF2FE7A5
:1002500084E89EE1215080409040E1F700C000001A
:10026000D2CF70D088F09F5790F0B92F9927B7510F
:10027000A0F0D1F0660F771F881F991F1AF0BA956A
:10028000C9F712C0B13081F077D0B1E0089574C0E1
:10029000672F782F8827B85F39F0B93FCCF3869560
:1002A00077956795B395D9F73EF4909580957095BD
:1002B00061957F4F8F4F9F4F0895E89409C097FB3A
:1002C0003EF490958095709561957F4F8F4F9F4F2D
:1002D0009923A9F0F92F96E9BB279395F695879571
:1002E00077956795B795F111F8CFFAF4BB0F11F434
:1002F00060FF1BC06F5F7F4F8F4F9F4F16C08823DB
:1003000011F096E911C0772321F09EE8872F762F10
:1003100005C0662371F096E8862F70E060E02AF051
:100320009A95660F771F881FDAF7880F969587953D
:1003300097F9089557FD9058440F551F59F05F3FA6
:1003400071F04795880F97FB991F61F09F3F79F0F7
:1003500087950895121613061406551FF2CF469579
:10036000F1DF08C0161617061806991FF1CF8695FB
:100370007105610508940895E894BB2766277727DF
:10038000CB0197F908950BD078C069D028F06ED0D2
:1003900018F0952309F05AC05FC01124EECFCADFD0
:1003A000A0F3959FD1F3950F50E0551F629FF00188
:1003B000729FBB27F00DB11D639FAA27F00DB11DE1
:1003C000AA1F649F6627B00DA11D661F829F22276A
:1003D000B00DA11D621F739FB00DA11D621F839FF1
:1003E000A00D611D221F749F3327A00D611D231FC7
:1003F000849F600D211D822F762F6A2F11249F5715
:1004000050408AF0E1F088234AF0EE0FFF1FBB1F37
:10041000661F771F881F91505040A9F79E3F5105D6
:1004200070F014C0AACF5F3FECF3983EDCF38695E2
:1004300077956795B795F795E7959F5FC1F7FE2B81
:10044000880F911D9695879597F9089597F99F675D
:1004500080E870E060E008959FEF80EC089500244C
:100460000A941616170618060906089500240A9419
:1004700012161306140605060895092E0394000C9F
:1004800011F4882352F0BB0F40F4BF2B11F460FF2E
:1004900004C06F5F7F4F8F4F9F4F0895F894FFCF39
:1004A000101010FC24BAAE66CEDEA4FEEE161EDAE4
:0604B00012ADF300020092
:00000001FF
